:100000000C948D000C94A6100C94AC000C94AC00D5
:100010000C94AC000C94AC000C94AC000C94890EC5
:100020000C94AC000C94AC000C94AC000C94AC00A0
:100030000C94AC000C94AC000C94AC000C94AC0090
:100040000C94AC000C94AC000C94AC000C94AC0080
:100050000C94AC000C94AC000C94AC000C94AC0070
:100060000C94AC000C94AC000C94AC000C94AC0060
:100070000C94AC000C94AC000C94AC000C94AC0050
:100080000C94AC000C94AC000C94AC00B80BDE0BE0
:10009000F20BF20B190C270C5E0CD70B1B0DB30BDC
:1000A000670C690C730C870C8B0CA10C3E0CAA0C12
:1000B000C70CCE0C1B0DD50CE10CF00CF70CFE0C94
:1000C000050D100D09021200010100C032090400E3
:1000D00000000000000012011001FF000008501D88
:1000E000E96000010102000112034B006500790084
:1000F0006D0061006E00360034001003480065009A
:100100006E006E0069006E0067002000420065000E
:100110006B0065006C000403090411241FBECFEFBF
:10012000D0E4DEBFCDBF18E0A0E0B1E0E6E4F1E34B
:1001300000E00BBF02C007900D92A23AB107D9F7B9
:100140002AE0A2EAB8E001C01D92A537B207E1F7A4
:100150000E94BA110C94A1180C94000020912B0954
:1001600030912C098091290990912A09AC014F5FA7
:100170005F4F50932A0940932909F901E80FF91FAD
:10018000808190E0089592B180912001809589232B
:1001900082B992B180912001892B82B9089592B1E0
:1001A00080912001892B82B992B1809120018095A4
:1001B000892382B90895CF93DF93DC01E0E0F0E07A
:1001C00090E8EA01888189232D913C9111972E0FA7
:1001D0003F1FEB01882329F08881892339F480E3CC
:1001E00006C08881892311F488E701C081E3E90111
:1001F000888396953196E830F10519F7ED91FC91D9
:10020000119710868D919C91DF91CF9108958091E7
:10021000E5089091E6089C012F5F3F4F3093E60878
:100220002093E5080E945F1890E00895682F809160
:10023000E3089091E4089C012F5F3F4F3093E4085E
:100240002093E3080E947D1880E090E00895CF920B
:10025000DF92EF92FF920F931F93CF93DF938C0166
:100260007B016A01C0E0D0E0D80112968D919C918B
:100270001397C817D907C0F4D8011896ED91FC91CF
:100280001997CE01880F991FE80FF91FB7018081D8
:1002900091810E94C514892B29F4F601D183C08372
:1002A00081E003C02196E0CF80E0DF91CF911F91E4
:1002B0000F91FF90EF90DF90CF900895CF92DF9253
:1002C000EF92FF920F931F93CF93DF93EC018B017B
:1002D0006A817B81888599856F5F7F4F660F771F65
:1002E0000E94C81399878887C884D984EA80FB80D4
:1002F000F80101900020E9F7CF0161E070E0801B78
:10030000910B0E948B12F701EE0FFF1FEC0DFD1DEC
:1003100091838083F80101900020E9F73197AF01C4
:10032000401B510B88859985EA81FB81EE0FFF1FE9
:10033000E80FF91FB801808191810E94CE148A8153
:100340009B8101969B838A838A819B810197DF91A0
:10035000CF911F910F91FF90EF90DF90CF90089574
:100360008F929F92AF92BF92EF92FF92CF93DF93C3
:10037000E0E0F0E0E12CF12CEC01AC81BD81EA166B
:10038000FB06C0F4EC01AA85BB85AE0FBF1F8D90A4
:100390009D90AD90BC90349684169506A606B7063F
:1003A00029F4F901F182E08281E005C0AFEFEA1A99
:1003B000FA0AE2CF80E0DF91CF91FF90EF90BF90FB
:1003C000AF909F908F900895CF92DF92EF92FF921F
:1003D000CF93DF93EC016A017B016C817D818A857B
:1003E0009B856F5F7F4F660F771F660F771F0E9499
:1003F000C8139B878A878A859B85EC81FD81EE0FD8
:10040000FF1FEE0FFF1FE80FF91FC082D182E282AB
:10041000F3828C819D8101969D838C838C819D814B
:100420000197DF91CF91FF90EF90DF90CF900895EB
:100430000F931F93CF93DF93EC018B016881798138
:100440008E819F816F5F7F4F660F771F0E94C81359
:100450009F838E838E819F81E881F981EE0FFF1F3C
:10046000E80FF91F11830083888199810196998390
:100470008883C801DF91CF911F910F910895FC01EE
:1004800020E030E08081918128173907C8F4A681E7
:10049000B781A901440F551FA40FB51F0D90BC9142
:1004A000A02D11968C91861308C086819781FC013E
:1004B000E40FF51F8081918108952F5F3F4FE2CFB8
:1004C00080E090E008950E943F0221E0892B09F02E
:1004D00020E0822F089520E030E0FC01408151812E
:1004E0002417350790F4DC011696ED91FC911797CF
:1004F000A901440F551FE40FF51F0190F081E02D75
:10050000438144832F5F3F4FE8CF0895CF93DF931C
:1005100067E070E081E090E00E948B12EC0162E005
:1005200070E081E090E00E948B129E838D83809129
:100530003706898380E48A8381E08B838C83CE01B4
:10054000DF91CF910895FF920F931F93CF93DF9385
:100550008C01F62E0E946302811109C06F2DC80123
:10056000DF91CF911F910F91FF900C943F020E9459
:100570008602EC01F982BC01C8010E941802CE017A
:10058000DF91CF911F910F91FF900895FC0161833E
:1005900008950F931F93CF93DF93EC018B01688134
:1005A00070E06F5F7F4F660F771F8D819E810E9485
:1005B000C8138D839E832881FC01E20FF11DE20F99
:1005C000F11D118300832F5F2883C801DF91CF9134
:1005D0001F910F910895FC012381248308950F93A7
:1005E0001F93CF93DF938C01C0E0D0E0F80120810E
:1005F00030E085819681C217D30764F49E01220FF3
:10060000331FFC01E20FF31F808191810E943F1391
:100610002196ECCF0E943F13C801DF91CF911F912B
:100620000F910C943F130F931F93CF93DF93EC0123
:1006300000E010E0288139818E819F810217130725
:1006400068F49801220F331FFC01E20FF31F808131
:1006500091810E94EF020F5F1F4FECCF0E943F136A
:1006600000E010E02A813B818885998502171307F5
:1006700068F49801220F331FFC01E20FF31F808101
:1006800091810E943F130F5F1F4FECCF0E943F13D9
:100690008A859B850E943F13CE01DF91CF911F91E8
:1006A0000F910C943F1365E070E081E090E00E94B0
:1006B0008B12FC0188E0808311828FEF8283838319
:1006C0001482CF0108959F92AF92BF92CF92DF9292
:1006D000EF92FF920F931F93CF93DF93EC0168E4A7
:1006E00076E00E945E0161E477E0CE010E945E0147
:1006F00067E377E0CE010E945E010E9486028C01D2
:1007000082E3F80181830E945303FC018CE0F82E00
:10071000F08212821382BF01C8010E94C902B8018F
:10072000CE010E9418020E9453036C018DE0F60175
:1007300080830E9486028C0183E2F8018183B601E6
:10074000C8010E94C902B801CE010E9418020E948D
:1007500086028C018AE2F80181830E945303FC0126
:10076000F08281E082831382BF01C8010E94C90226
:100770009AE0E92EF12C2FE0922E35E2A32E45E0EF
:10078000B42E58EEC52E63E0D62E0E945303FC0112
:100790009082A382BC01C8010E94C9020E94530337
:1007A000FC01B082C282D382BC01C8010E94C9028E
:1007B000F1E0EF1AF10849F70E945303FC018CE0C5
:1007C000808382E082831382BF01C8010E94C90234
:1007D000B801CE010E9418020E9486028C018BE3B0
:1007E000F80181830E945303FC0186E18083128219
:1007F0001382BF01C8010E94C902B801CE010E9444
:10080000180281E0DF91CF911F910F91FF90EF903F
:10081000DF90CF90BF90AF909F9008950F931F935C
:10082000CF93DF93EC018B01CB010E94DD14982F55
:10083000991F9927991F9983982F90769C838F7180
:100840008883C8010E94DD148A83C8010E94DD14D8
:100850008B83DF91CF911F910F910895CF92DF92FB
:10086000EF92FF920F931F93CF93DF936C017B0165
:10087000CB010E94DD14F6018383C7010E94DD14C1
:1008800000E010E0EC01DD270C171D0764F40E9466
:100890005303BC01C6010E94C902B7010E940E04A5
:1008A0000F5F1F4FF1CFDF91CF911F910F91FF90FD
:1008B000EF90DF90CF9008950C943F1364E070E0C8
:1008C00081E090E00C948B12CF93DF936EE070E0A8
:1008D00081E090E00E948B12EC0162E070E081E028
:1008E00090E00E948B129F838E83198618861B8648
:1008F0001A860E945E049D878C87198218821B824B
:100900001A821D821C82CE01DF91CF9108950F9330
:100910001F93CF93DF93EC018B01CB010E94DD1479
:100920008883C8010E94DD148983C8010E94DD14F8
:100930008A83C8010E94DD148B83DF91CF911F91C0
:100940000F9108958F929F92AF92BF92CF92DF92B4
:10095000EF92FF920F931F93CF93DF93CDB7DEB744
:10096000D0510FB6F894DEBF0FBECDBF5C018B0136
:10097000FC01848595850E948704CE0101964C0177
:10098000C8010E94DD14F82E80913806F81609F48B
:1009900063C0809136068F1116C064017601E81895
:1009A000F908C8010E94DD14882321F0F601819323
:1009B0006F01F4CFF401EE0DFF1D1082B401C501EB
:1009C0000E945E01DDCF80913506F81239C0C80162
:1009D0000E94DD147C01C8010E94DD146C01C80175
:1009E0000E94DD14A601DD0C660B770B762F652FB8
:1009F000542F4427092E000CAA0BBB0BDC019927AE
:100A00008827842B952BA62BB72B6701FF0CEE08AC
:100A1000FF08C82AD92AEA2AFB2AC8010E94DD1445
:100A2000AC01990F660B770B742F66275527442767
:100A30004C295D296E297F29C5010E94E401A0CFC0
:100A40000E948602BC01C5010E941802FC01F182CD
:100A5000B8010E942E0494CF81E0D05F0FB6F894C5
:100A6000DEBF0FBECDBFDF91CF911F910F91FF90E1
:100A7000EF90DF90CF90BF90AF909F908F900895B0
:100A80000F931F93CF93DF9300D0CDB7DEB78C01C8
:100A9000CB0169837A830E94DD14909139066981C4
:100AA0007A8198130BC0CB0169837A830E94DD148D
:100AB00090913A0669817A81981759F090E00E94E6
:100AC000961580E00F900F90DF91CF911F910F91BD
:100AD0000895C8010F900F90DF91CF911F910F9152
:100AE0000C94A2040C943F13F8949CE088E10FB698
:100AF000F894A895809360000FBE90936000FFCF9C
:100B0000EEE3F9E081E08083118208950E94800580
:100B1000EEE3F9E0128213821482158208950E9496
:100B2000860580911D0180937300E8E6F0E08081E6
:100B300088608083789408950FB6F894A895809182
:100B40006000886180936000109260000FBE8FEF9C
:100B500081B980EC82B989E88AB980EF8BB90C94AD
:100B60008F0580E090E0FC01EE0FFF1FEE0FFF1FEE
:100B7000EC57F64F1182108201968031910599F75A
:100B80000895CF93DF93882339F026E230E0A8E27E
:100B9000B0E0C7E2D0E006C023E230E0A5E2B0E07A
:100BA000C4E2D0E098E0899FF0011124E62BEE0F1B
:100BB000FF1FEE0FFF1FEC57F64F31832083628338
:100BC00043838881962F9095892388838C91682B05
:100BD0006C93DF91CF910895F8940E948610519AFA
:100BE0002FEF89E698E1215080409040E1F700C066
:100BF00000005198789410922C0910922B090895B6
:100C000080E090E0FC01EB5FF54F8083019680343B
:100C10009105C1F7089585B7806885BF85B780685D
:100C200085BF08959BB180912101892B8BB99BB120
:100C300080912101809589238BB908959BB1809182
:100C40002301892B8BB98AE18A95F1F700C09BB10A
:100C500080912301809589238BB90895CF92DF92EB
:100C6000FF920F931F93CF93DF931F92CDB7DEB701
:100C70000E941206C12CD12C80E0FF24F39486013F
:100C8000085F1F4F29B1909122019223F601EC5386
:100C9000F64F911103C0F08281E001C01082898378
:100CA0000E941E069FEFC91AD90A89810C151D05DD
:100CB00049F768010034110511F70F90DF91CF91CA
:100CC0001F910F91FF90DF90CF900895E82FF0E0F3
:100CD000EC5BF64F9081911111C090911F0166233A
:100CE00011F0892B02C09095892390912001892BC6
:100CF00082B9E0913209F091330909940895CF93B4
:100D00009BB180911E01809589238BB98FE99FE06B
:100D10000197F1F700C000009BB180911E01892B63
:100D20008BB9C0E060E08C2F0E946606CF5FC034B4
:100D3000C9F7CF910895CF939BB180911E01892B64
:100D40008BB98FE99FE00197F1F700C000009BB1DC
:100D500080911E01809589238BB9C0E060E08C2FC3
:100D60000E946606CF5FC034C9F7CF910895EF9215
:100D7000FF920F931F93CF93DF931F92CDB7DEB7F0
:100D8000182F062F90E09C012C5B364F7901F9015A
:100D90008081882319F0808184131DC0F701808130
:100DA000811106C0602F812F49830E946606498108
:100DB000011101C040E0F7014083808181110BC027
:100DC000602F812F0F90DF91CF911F910F91FF9096
:100DD000EF900C9466060F90DF91CF911F910F91C9
:100DE000FF90EF900895CF93DF93C0E0D0E0FE0135
:100DF000EE0FFF1FEE0FFF1FEC57F64F8081918122
:100E0000892BB1F0A081B1819C918281892321F449
:100E1000838142E061E00AC0A381B0E0AC5BB64FE1
:100E20008C91823029F4838142E060E00E94B70611
:100E30002196C031D105D9F6DF91CF910895CF9396
:100E4000DF93C0E0D0E0FE01EC53F64F6081FE017D
:100E5000EB5FF54F80810E9466062196C034D10574
:100E600091F7DF91CF910895CF93DF931F92CDB784
:100E7000DEB78983898161E00E9466062FEF89EFE2
:100E800090E0215080409040E1F700C0000089814F
:100E900060E00F90DF91CF910C946606CF93DF93C3
:100EA0001F92CDB7DEB78983E981F0E0EC53F64FAE
:100EB00080810F90DF91CF910895CF93DF931F92A0
:100EC000CDB7DEB78983E981F0E0EC53F64F90812E
:100ED00081E089270F90DF91CF910895CF93DF9321
:100EE0001F92CDB7DEB78983998181E0903408F0F5
:100EF00080E00F90DF91CF910895CF93DF931F9201
:100F0000CDB7DEB789838981803410F080E021C0BD
:100F10000E942E068823D1F3E981F0E0EC53F64FCE
:100F20008081882399F32FEF89EF90E02150804052
:100F30009040E1F700C000000E942E06882331F0A7
:100F4000E981F0E0EC53F64F808102C080E090E050
:100F500081700F90DF91CF910895CF93DF931F920F
:100F6000CDB7DEB789838981803410F080E01BC063
:100F70000E942E06E981F0E0EC53F64F808181114A
:100F8000F5CF2FEF89EF90E0215080409040E1F7BE
:100F900000C000000E942E06E981F0E0EC53F64FFD
:100FA000908181E089270F90DF91CF9108958F92F2
:100FB0009F92AF92BF92CF92DF92FF920F931F93B7
:100FC000CF93DF93EC018C01FE0101900020E9F743
:100FD0003197EC1BFD0BC8018C1B9D0B8E179F07D7
:100FE00008F04AC0D801ED918D01F0E0CF01880FE3
:100FF000991FE80FF91FEC5DFE4FC2808080918041
:101000005401D12CC501881999098C159D05E4F668
:10101000F50181915F01982F907C903849F461E04F
:101020008F730E9466068FE99FE00197F1F70AC06F
:10103000903459F460E08F730E946606AFE9BFE018
:101040001197F1F700C00000DDCF903CD9F68F7307
:10105000F82E80913C09F81209C0BFEFE9EFF0E0EB
:10106000B150E040F040E1F700C000008F2D0E9439
:101070003407F0923C09C6CFDF91CF911F910F91B9
:10108000FF90DF90CF90BF90AF909F908F9008958A
:10109000CF93DF93CDB7DEB7D2500FB6F894DEBF53
:1010A0000FBECDBF9E012B5F3D4FF9014191519184
:1010B0009F0160E072E0CE0101960E945D15CE01B5
:1010C00001960E94D707DE5F0FB6F894DEBF0FBE11
:1010D000CDBFDF91CF910895CF92DF92FF920F9312
:1010E0001F93CF93DF931F92CDB7DEB780E090E0E0
:1010F000FC01E951F74F1082019680349105C1F748
:1011000005EE17E020E090E0223048F0F80131973A
:101110008081803221F4F8018081803289F0FF24BF
:10112000F394F90EC92ED12CF801808190E0298327
:101130000E94AD14F601E951F74F80839F2D29815C
:101140002F5F0F5F1F4F2132F9F60F90DF91CF9184
:101150001F910F91FF90DF90CF900895CF93DF9371
:1011600000D0CDB7DEB787E098E09A83898344E268
:1011700050E065E270E0CE0101960E94DB009F9393
:101180008F9380E198E09F938F930E94480847E2F5
:1011900050E068E270E0CE0101960E94DB009F9370
:1011A0008F9386E198E09F938F930E9448080FB633
:1011B000F894DEBF0FBECDBF0F900F90DF91CF919F
:1011C0000895FC0184B1808385B1818387B18283D6
:1011D00088B183830895FC01808184B9818185B9B8
:1011E000828187B9838188B90895FC019181923009
:1011F00089F118F4992349F03CC0933031F09430D0
:10120000C1F581E080933D0934C090933109868116
:10121000978190932E0980932D09828193819093D9
:101220002809809327091092300910922F09809184
:101230002B0990912C09892BF1F460912D09709163
:101240002E0981E090E00E948B1290932C098093EC
:101250002B0911C0E7EEF8E0F093560AE093550A27
:1012600001900020E9F73197E75EF84081E08E0FAA
:10127000089580E008958FEF089540912D095091D1
:101280002E092EE031E061E070E080912B09909111
:101290002C090E941B1540912D0950912E0921E027
:1012A0008417950709F020E0209339090895CF931A
:1012B0000E942E0680E090E0C82FFC01EC53F64F10
:1012C0002081222331F08C2F0E94AD078823D9F38F
:1012D00006C001968034910579F78FEF01C08C2FFD
:1012E000CF9108950F931F93CF93DF93EB01188253
:1012F0009F938F930E9448080F900F900DE118E084
:101300000E9457098F3FE1F3FE0101900020E9F7A9
:101310003197EC1BEF3311F41882E0E09E012E0FA1
:10132000311DF90180831182883069F48AE898E0E0
:101330009F938F930E9448080F900F90DF91CF9159
:101340001F910F9108951F930F930E9448080F90CB
:101350000F90D6CFCF93DF930E9457098F3F09F4A8
:101360003FC0E3EAF8E001900020E9F73197E35A43
:10137000F840EF3319F41092A308E0E0F0E0ED55E7
:10138000F74F80831182E3EAF8E001900020E9F74B
:101390003197BF01635A7840962FA0913709B091D9
:1013A000380923EA38E0169680E0ED01891758F4F1
:1013B000F90151919F014D91541719F01092A30812
:1013C0000FC08F5FF3CFDE010D900020E9F711977A
:1013D000AC1BBD0BFB01FF2781E0EA17FB0709F0FF
:1013E00080E0DF91CF910895CF93DF9368E470E0C0
:1013F00081E090E00E948B12EC010E945E049D83CC
:101400008C83CE01DF91CF9108950F931F93FC0140
:1014100081E0008111812281338140912906509120
:101420002A0660912B0670912C06041715072607D3
:10143000370709F080E01F910F9108954091290628
:1014400050912A0660912B0670912C06FC01408376
:101450005183628373831682EA5BFF4F118210828D
:101460000895CF93DF93EC01809127069091280691
:101470000E946718688379838A839B83DF91CF9169
:101480000895EF92FF920F931F93CF93DF938C01F8
:10149000C0912706D0912806FC01E480F580CE019A
:1014A00004960E945F18F7018083F801E480F580BC
:1014B000CE0105960E945F18F7018183F801E48050
:1014C000F580CE0106960E945F18F7018283F8012D
:1014D00004811581CE0107960E945F18F80183836D
:1014E000DF91CF911F910F91FF90EF900895809120
:1014F0003709909138090E94410AE0913709F0912B
:101500003809848195810C94EB08609127067091CD
:1015100028066A5F7F4F40E450E006960C944F180F
:1015200008954091290650912A0660912B067091EA
:101530002C0680912706909128060C948F180F9303
:101540001F93CF93DF938C01C0912706D09128067B
:10155000DC011496ED91FC9115976081CE01049603
:101560000E947D18D8011496ED91FC911597618128
:10157000CE0105960E947D18D8011496ED91FC913C
:1015800015976281CE0106960E947D18D8011496A7
:10159000ED91FC9115976381CE010796DF91CF9174
:1015A0001F910F910C947D18E0913709F091380943
:1015B000848195810E94E1088091370990913809D2
:1015C0000C949F0A60912706709128066A5F7F4FEE
:1015D00040E450E006960C946D18CF92DF92EF92A3
:1015E000FF920F931F93CF93DF93CDB7DEB7C05811
:1015F000D1090FB6F894DEBF0FBECDBF8E010F5BD1
:101600001F4FD8011D921D921D921C921397FE012F
:10161000EB5BFF4F8CE3DF01282F1D922A95E9F742
:1016200019821A821B821C82E054F109DF011D928B
:101630008A95E9F7B8018BE298E00E947209FE01F1
:1016400031966F01BF0180E498E00E947209F801B1
:1016500001900020E9F731977F01E01AF10AF601C5
:1016600001900020E9F73197EC19FD09EE16FF060D
:1016700009F040C0B601C8010E94C514892BD1F5FC
:101680008091370990913809EA94EF2839F4D8010C
:101690002C91283019F4FC01168206C040E450E079
:1016A000B80106960E94CE148091370990913809AE
:1016B0000E94E20AA0913709B09138091696FD01FF
:1016C00001900020E9F73197EA1BFB0B329718F4E1
:1016D00083E298E002C08FE198E09F938F9386E5C4
:1016E00098E09F938F930E9448080F900F900F905F
:1016F0000F9008C088E698E09F938F930E94480857
:101700000F900F90C058DF4F0FB6F894DEBF0FBE9A
:10171000CDBFDF91CF911F910F91FF90EF90DF90A0
:10172000CF900895FF920F931F93CF93DF938C0177
:10173000DB0111968C911197882329F0C8E2D0E043
:1017400027E230E004C0C5E2D0E024E230E0FC90C3
:101750004F2D50E04C31510508F06DC1FA01EA5BA4
:10176000FF4F0C94821213968C918093040A63C1EC
:1017700012964C911297942F50E090FD03C09695CD
:101780005F5FFBCF13968C911397892301C0880F5D
:101790005A95EAF798814095492348839881892B87
:1017A0008883F901908112968C91892BC8C0F90128
:1017B000908112968C911297892B42C09881129633
:1017C0008C9112979823F9014081482B40833881EE
:1017D00012962C9120952323288328818927822BF8
:1017E000888329C112965C9112979881452F4923CD
:1017F000F2E0FF1202C091E001C09FEF852F60E090
:1018000080FD04C0869546956F5FFACF940F8923BB
:1018100001C0880F6A95EAF7F9019081952B9083B2
:10182000288112969C919095922398839881892B78
:10183000D7CFF901908112968C91129780958923C8
:101840008083988112968C9180958923C9CF1296B6
:101850008D919C911397092E000CAA0BBB0B00973E
:10186000A105B10509F4E7C0EFE9FFE03197F1F711
:1018700000C000000197A109B109F1CFF8018285EC
:1018800093851296ED91FC911397EE0FFF1FEE0FCB
:10189000FF1FE80FF91F80819181A281B38100971A
:1018A000A105B10509F4C7C0EFE9FFE03197F1F7F1
:1018B00000C000000197A109B109F1CF13968C91E6
:1018C000DF91CF911F910F91FF900C94290E61E051
:1018D00001C060E013968C91DF91CF911F910F9121
:1018E000FF900C946606F801808591851296ED9123
:1018F000FC911397EE0FFF1FE80FF91F8081918174
:10190000DF91CF911F910F91FF900C94D70781E049
:1019100080933D0990C01296EC911297F0E0EB5F36
:10192000F54F80811396CC911397D0E0CB5FD54FC4
:10193000988190831396EC91F0E0EB5FF54F8083F4
:101940007AC013968C91DF91CF911F910F91FF90E8
:101950000C94340713968C91811109C08FE796E09F
:10196000909335098093340983EC90E00BC081306B
:1019700009F061C08BE996E09093350980933409B2
:101980008FEC90E0909333098093320954C0DF913B
:10199000CF911F910F91FF900C94D40ADF91CF91BA
:1019A0001F910F91FF900C94770A13964C91139707
:1019B00012966C91DF91CF911F910F91FF900C9433
:1019C000C10587EE98E09F938F9388E198E09F93FD
:1019D0008F930E9448080F900F900F900F902BC08C
:1019E000DF91CF911F910F91FF900C94AE08DF9182
:1019F000CF911F910F91FF900C94F00EDF91CF913A
:101A00001F910F91FF900C94ED0A80913A099091EB
:101A10003B09DF91CF911F910F91FF900C94E1084A
:101A200080913A0990913B09DF91CF911F910F91DD
:101A3000FF900C94EB08DF91CF911F910F91FF90D5
:101A40000895AF92BF92CF92DF92EF92FF920F93E1
:101A50001F93CF93DF93EC015B0100E010E08881DE
:101A600099810817190708F045C0EE81FF816801C8
:101A7000CC0CDD1CEC0DFD1D0190F081E02D918161
:101A800080913706981329C0E12CF12C1AC0EE8101
:101A9000FF81EC0DFD1D0190F081E02D0580F681A8
:101AA000E02DC701880F991FE80FF91F6081718130
:101AB000CE010E94920BA114B10491F48FEFE81AA9
:101AC000F80AEE81FF81EC0DFD1D0190F081E02D03
:101AD000808190E0E816F906D4F20F5F1F4FBFCF68
:101AE000C501EFE9FFE03197F1F700C00000019771
:101AF000C1F7E4CFDF91CF911F910F91FF90EF904D
:101B0000DF90CF90BF90AF900895CF93DF930E9466
:101B10006404EC0110922A091092290960E071E036
:101B20000E944005882339F06091270970912809A7
:101B3000CE010E94210DCE01DF91CF910C941303B1
:101B400040912B0950912C09FC0170E0A0912F09C4
:101B5000B091300920912D0930912E09A217B307B9
:101B6000C8F49F01281B390B261737079CF4A09156
:101B70002F09B0913009A40FB51F21912C9320910A
:101B80002F09309130092F5F3F4F30933009209358
:101B90002F09DCCF20912F093091300980912D0938
:101BA00090912E0928173907C8F0809131098111C9
:101BB00003C00E94850D06C080913109833011F465
:101BC0000E943D0980912B0990912C090E943F139E
:101BD00010922C0910922B0981E0089580E008955D
:101BE0000F931F93CF93DF93EC0100E010E0888107
:101BF00090E0081719070CF5ED81FE81C801880FE8
:101C0000991FE80FF91F60817181FB01848188238E
:101C100059F0803421F48A81803461F405C0803623
:101C200049F48A81803631F48091450A9091460AC0
:101C30000E94920B0F5F1F4FDACF8A81803411F020
:101C400080E401C080E68A83DF91CF911F910F91DC
:101C500008951F93CF93DF93182FC0E0D0E0E09159
:101C6000450AF091460A80819181C817D90790F4FE
:101C70000680F781E02DCE01880F991FE80FF91F2C
:101C800080819181FC012181211302C00E94F00D0D
:101C90002196E5CFDF91CF911F9108958091400962
:101CA0008330A1F028F4813041F0823051F0089562
:101CB0008430C9F08530D9F00895809141090C94A1
:101CC000290E8091410941E061E004C08091410901
:101CD00041E060E00E94B7068FE99FE00197F1F7CD
:101CE00000C000000895809141090C943407809150
:101CF00042099091420940914109977061E070E07A
:101D000001C0660F9A95EAF783FB882780F90C9447
:101D1000C1051F920F920FB60F9211240BB60F92AE
:101D20002F933F934F935F936F937F938F939F93E3
:101D3000AF93BF93EF93FF9399B180911D018923D6
:101D4000E1F599B180911C01892339F090913E0908
:101D500080913F09892B80933F0980913E09880F2C
:101D600080933E0980913E09811127C080914309EB
:101D700081110DC080913F0980934009E091400995
:101D8000F0E0E15DF94F8081809343090BC0E09161
:101D90004309E150E0934309F0E080913F09E25CA0
:101DA000F64F838380914309811105C00E944E0E36
:101DB0000E94860502C00E948005FF91EF91BF91AD
:101DC000AF919F918F917F916F915F914F913F91D3
:101DD0002F910F900BBE0F900FBE0F901F90189574
:101DE000E0913709F09138098681882339F08BEF2B
:101DF0000E94290E82E08093A20808958CE898E062
:101E00009F938F930E9448080F900F9008958AEF38
:101E10000E94290E1092A2080895CF93DF93EC013F
:101E20008C81882349F081508C83811105C0CE01BB
:101E30000E94F00D8B818C83DF91CF9108958A5B96
:101E40009F4FFC0160817181809127069091280647
:101E50008A5B9F4F0C949B188091370990913809A9
:101E6000FC01EA5BFF4F20912D0630912E06318355
:101E700020830E941F0F0E947405CF93DF93EC0113
:101E80000E94910ACE010E949F0ACE010E94E20A9E
:101E9000CE01DF91CF910C941F0FCF93DF93EC0114
:101EA0000E94310A4091290650912A0660912B0622
:101EB00070912C0688819981AA81BB8148175907A6
:101EC0006A077B0741F4CE010E94410ACE01DF91EF
:101ED000CF910C94850ACE010E941E0ACE01DF919B
:101EE000CF910C943D0FCF93DF93EC018C819D81BA
:101EF0000E943F13CE01DF91CF910C943F13CF93FB
:101F0000DF936091570A635067FDA7C08091540A20
:101F1000CCE0D0E0C81BD109C55AD54F8091530AF7
:101F20008D3209F088C0683009F095C083EC809349
:101F3000470A8AE580933C06109236092881822F51
:101F4000807639F0CE010E94F5088F3F09F462C017
:101F500068C08A811092500A998191110BC02F712B
:101F600019F481E08093500A1092510A20E53AE07A
:101F700082E04BC0953019F48093580A38C09630EF
:101F800081F59B81913019F486ED90E01FC092306D
:101F900019F484EC90E01AC09330F1F4811108C078
:101FA00086E191E09093560A8093550A84E015C02B
:101FB000813041F48AEF90E09093560A8093550A5D
:101FC0008CE10BC0823041F488EE90E09093560A89
:101FD0008093550A82E101C080E090E49093360935
:101FE00020C0983079F0993031F480935A0A20E576
:101FF0003AE080E00AC081E09A3009F080E020E514
:102000003AE003C02AE53AE081E03093560A209393
:10201000550A07C0988197FD8E8190E89093360904
:1020200007C09F81911104C09E81981708F4892FE1
:1020300080933B0610C08091360987FF0CC0CE010B
:102040000E94A00D8F3F21F48EE180933C0603C0D7
:10205000811110923B061092570A80913C0684FF32
:1020600048C080913B068F3F09F443C0C82F893098
:1020700008F0C8E08C1B80933B069091470A88E8E3
:1020800089278093470ACC2331F14091550A50911A
:10209000560A8091360986FF0AC0A8E4BAE0FA0120
:1020A0009C2F84918D9331969150D9F708C0DA0115
:1020B000E8E4FAE09C2F8D9181939150E1F72FEFA6
:1020C0002C0F30E02F5F3F4FCA01820F931F909378
:1020D000560A8093550A6C2F88E49AE00E94A21059
:1020E00064E06C0F6C3019F08FEF80933B066093C7
:1020F0003C0684E199B1967031F48150D9F7109281
:10210000580A1092520ADF91CF910895E9E6F0E063
:10211000808182608083E89A0895A82FB92F80E09B
:1021200090E041E050EA609530E009C02D918227AF
:102130009795879510F084279527305EC8F36F5FD9
:10214000A8F30895EADF8D939D930895CF93CFB7B9
:10215000CF93DF93C395499BE9F7499B0BC0499BFC
:1021600009C0499B07C0499B05C0499B03C0499BC7
:1021700001C089C06F93C091540ADD27C55AD54F5D
:102180002F9365E5499B03C02F916F91E6CF0F9385
:102190001F934F9320E040E15F9309B1067001FB6C
:1021A00027F93F9350E03BE039C0167040642F7729
:1021B000012F5F5F1EC0406819B116702F77525013
:1021C0001FC0406409B12F770670D1F15F5F00C076
:1021D00023C0406219B12F77167091F15F5F00C084
:1021E00025C006701027515012F45D5F0000115099
:1021F00027952C3F19B1C8F6167001270150279575
:102200002C3FC8F64227499309B1067010274F7337
:10221000115027952C3FA8F64695469519B1167092
:1022200079F00127015027952C3F98F66B5A60F3FF
:10223000315009B1B0F600C011E01CBB002717C037
:102240003B503195C31BD04011E01CBB0881033CBF
:10225000F9F00B34E9F02091520A1981110F121391
:10226000EDCF093651F10D3211F0013E39F70093EF
:10227000590A3F915F914F911F910F912F916F914B
:10228000CCB3C0FD67CFDF91CF91CFBFCF91189571
:102290002091590A222369F31091570A112339F525
:1022A00034303AF13093570A2093530A1091540A6C
:1022B0003BE0311B3093540A1CC00091570A013097
:1022C000B4F40AE530913C0634FD14C000933C069A
:1022D000C7E4DAE013C0052710E000C000000BB926
:1022E0001AC0052710E0221F1DC010E021C04AE5DA
:1022F00002C032ED432FC4E1D0E032E01AB11660E3
:10230000599A0BB11AB956E020E865E320FF05277A
:102310000BB9279517951C3FF0F66695B8F7B1F7FE
:1023200020FF05270BB9279517951C3FD0F6279559
:10233000179517FF052700001C3F0BB9B0F6299130
:102340003A9519F7097F1091580A110FC651D040DC
:102350000BB911F01093520A11E01CBB02601AB1C4
:10236000197F402F497F54E05A95F1F70BB91AB9FC
:102370004BB97FCF0E949C050E9400060E94B105C8
:102380000E946C088FE08093040A10923D0910921D
:1023900039098BE996E090933509809334098FECE5
:1023A00090E090933309809332090E9464049093E3
:1023B000460A8093450A6EE071E00E944005811153
:1023C00006C08091450A9091460A0E946303E091FD
:1023D0003409F0913509099560E070E08091450A73
:1023E0009091460A0E94210D0E94EC050E94F4097A
:1023F00090933809809337090E944D0F0E945E0424
:1024000090933B0980933A090E94E10811E001E0B2
:102410000E947F0F80913D09811104C0809139098C
:10242000882399F02FEF84E39CE021508040904076
:10243000E1F700C0000080913D0981110E942C0F3E
:102440008091390981110E9474050E94F3068091E0
:10245000A2088130C1F020F0823009F44BC0D8CFFF
:102460008091040A0E947D07882351F08091450ADB
:102470009091460A0E946B020093A20811E0C8CF17
:102480000E941F07C5CF8091040A0E94AD078111E9
:1024900003C0C0E0D0E024C0112321F08091040AE1
:1024A0000E9434071092A208B3CF0680F781E02D76
:1024B000CE01880F991FE80FF91FE080F180F70126
:1024C00081810E947D07882351F0C7010E940D0F72
:1024D000F70181810E94AD078823D1F310E0219696
:1024E000E091450AF091460A80819181C817D90789
:1024F000E0F28ECF0E94AA09882309F489CF0E94B6
:10250000070F86CFEE0FFF1F0024001C0BBE0790A5
:10251000F691E02D09940F931F93CF93DF93869F3D
:102520008001879F100D969F100D1124C8010E94F5
:10253000A712EC01009729F0A80160E070E00E946A
:10254000BE14CE01DF91CF911F910F9108950F938B
:102550001F93CF93DF938230910510F482E090E0D7
:10256000E091730AF091740A20E030E0A0E0B0E05E
:10257000309719F140815181028113814817590721
:10258000C8F08417950769F4109731F012960C93F0
:10259000129713961C9327C00093730A1093740A22
:1025A00022C02115310519F04217530718F49A017A
:1025B000BD01EF01DF01F801DBCF21153105F9F095
:1025C000281B390B2430310580F48A819B816115E9
:1025D000710521F0FB019383828304C09093740AF8
:1025E0008093730AFE01329644C0FE01E20FF31F8E
:1025F0008193919322503109398328833AC02091E5
:10260000710A3091720A232B41F420913F063091D8
:1026100040063093720A2093710A20913D06309152
:102620003E062115310541F42DB73EB740914106D4
:1026300050914206241B350BE091710AF091720A09
:10264000E217F307A0F42E1B3F0B2817390778F089
:10265000AC014E5F5F4F2417350748F04E0F5F1FE8
:102660005093720A4093710A8193919302C0E0E003
:10267000F0E0CF01DF91CF911F910F910895CF939B
:10268000DF93009709F481C0FC0132971382128214
:10269000A091730AB091740A109781F4208131815E
:1026A000820F931F2091710A3091720A28173907FF
:1026B00051F5F093720AE093710A67C0ED0120E0D2
:1026C00030E0CE17DF0740F44A815B819E0141155F
:1026D0005105F1F0EA01F5CFD383C28340815181E6
:1026E000840F951FC817D90759F488819981840FE1
:1026F000951F0296918380838A819B819383828335
:102700002115310529F4F093740AE093730A3DC052
:10271000E901FB83EA8349915991C40FD51FEC1756
:10272000FD0761F480819181840F951F0296E90174
:1027300099838883828193819B838A83E0E0F0E0A0
:1027400012968D919C911397009719F0FD01DC0171
:10275000F7CF8D919C9111979D012E5F3F4F820F76
:10276000931F2091710A3091720A2817390769F472
:10277000309729F41092740A1092730A02C01382DF
:102780001282B093720AA093710ADF91CF910895DB
:102790006F927F928F929F92AF92BF92CF92DF9271
:1027A000EF92FF920F931F93CF93DF93EC0100976B
:1027B00089F4CB01DF91CF911F910F91FF90EF90A2
:1027C000DF90CF90BF90AF909F908F907F906F9051
:1027D0000C94A712FC01E60FF71F9C01225031094F
:1027E000E217F30708F4A8C0D9010D911C911197C5
:1027F00006171707B0F00530110508F49BC0C80193
:1028000004978617970708F495C002501109061B14
:10281000170B019311936D937C93CF010E943F138B
:1028200089C05B01A01AB10A4C01800E911EA091D3
:10283000730AB091740A612C712CE12CF12C109761
:1028400009F446C08D919C911197A815B905B1F571
:102850006C0142E0C40ED11CCA14DB0478F14C01B7
:102860008A189B08640142E0C40ED11C1296BC90E9
:1028700012971396AC91B5E0CB16D10440F0B2821A
:10288000A38391828082D9016D937C9309C00E5FEE
:102890001F4F800F911FF90191838083EB2DFA2F39
:1028A000E114F10431F0D7011396FC93EE931297E3
:1028B00041C0F093740AE093730A3CC0681679062D
:1028C00008F43C017D0112960D90BC91A02DB7CF6C
:1028D0008091710A9091720A88169906E1F4661641
:1028E0007706C8F480913D0690913E06009741F42A
:1028F0008DB79EB74091410650914206841B950BBF
:10290000E817F907C8F4F093720AE093710AF90125
:10291000718360830FC0CB010E94A7127C010097D6
:1029200059F0A801BE010E94B514CE010E943F13C8
:10293000C70104C0CE0102C080E090E0DF91CF91DA
:102940001F910F91FF90EF90DF90CF90BF90AF90CD
:102950009F908F907F906F9008959111089581546A
:102960008A5108F4805E855A0895FB01DC0102C09B
:1029700001900D9241505040D8F70895DC0101C0FC
:102980006D9341505040E0F70895FB01DC018D91BB
:10299000019080190110D9F3990B0895FB01DC0116
:1029A0004150504048F001900D920020C9F701C0FD
:1029B0001D9241505040E0F70895CF93DF93EC0112
:1029C0002B8120FF33C026FF0AC02F7B2B838E81F3
:1029D0009F8101969F838E838A8190E029C022FF88
:1029E0000FC0E881F9818081082E000C990B0097B7
:1029F00019F420622B831AC03196F983E8830EC044
:102A0000EA85FB85099597FF09C02B81019611F096
:102A100080E201C080E1822B8B8308C02E813F8140
:102A20002F5F3F4F3F832E83992702C08FEF9FEF89
:102A3000DF91CF9108958F929F92AF92BF92CF92E4
:102A4000DF92EF92FF920F931F93CF93DF935B017F
:102A50004A017901D90113962C9121FF1DC0C0E0D4
:102A6000D0E0C815D905D9F08C016C01CA0CDB1C6B
:102A7000C8010C151D0571F00F5F1F4FD701189687
:102A8000ED91FC911997B701DC018C910995892B87
:102A900079F305C02196E5CF80E090E001C0CE013A
:102AA000DF91CF911F910F91FF90EF90DF90CF902A
:102AB000BF90AF909F908F9008950F931F93CF93E7
:102AC000DF93CDB7DEB72E970FB6F894DEBF0FBEFB
:102AD000CDBF8C01FA0186E08C831A83098377FFCE
:102AE00002C060E070E8CB0101979E838D83A9014D
:102AF000BF01CE0101960E94AF154D815E8157FD49
:102B00000AC02F813885421753070CF49A01F80147
:102B1000E20FF31F10822E960FB6F894DEBF0FBEA1
:102B2000CDBFDF91CF911F910F910895FB012381BC
:102B300020FF12C026FD10C08F3F3FEF930761F0CA
:102B400082832F7D206423832681378121503109A0
:102B500037832683992708958FEF9FEF08952F924B
:102B60003F924F925F926F927F928F929F92AF921D
:102B7000BF92CF92DF92EF92FF920F931F93CF936A
:102B8000DF93CDB7DEB72C970FB6F894DEBF0FBE3C
:102B9000CDBF6C017B018A01FC0117821682838103
:102BA00081FFBEC1CE0101964C01F6019381F70170
:102BB00093FD859193FF81917F01882309F4ACC136
:102BC000853239F493FD859193FF81917F018532A0
:102BD00029F4B60190E00E94C117E7CF512C312CA7
:102BE00020E02032A0F48B3269F030F4803259F0CA
:102BF000833269F420612CC08D3239F0803339F48E
:102C0000216026C02260246023C0286021C027FDE7
:102C100027C030ED380F3A3078F426FF06C0FAE0CE
:102C20005F9E300D1124532E13C08AE0389E300D64
:102C30001124332E20620CC08E3221F426FD6CC18B
:102C4000206406C08C3611F4206802C0883641F436
:102C5000F70193FD859193FF81917F018111C1CF90
:102C6000982F9F7D9554933028F40C5F1F4F9FE35E
:102C700099830DC0833631F0833771F0833509F0C5
:102C80005BC022C0F801808189830E5F1F4F4424FE
:102C90004394512C540115C03801F2E06F0E711CA1
:102CA000F801A080B18026FF03C0652D70E002C04E
:102CB0006FEF7FEFC5012C870E94B6172C018301AF
:102CC0002C852F77222E17C03801F2E06F0E711C71
:102CD000F801A080B18026FF03C0652D70E002C01E
:102CE0006FEF7FEFC5012C870E94AB172C012C855D
:102CF0002068222E830123FC1BC0832D90E0481600
:102D00005906B0F4B60180E290E00E94C1173A94EF
:102D1000F4CFF50127FC859127FE81915F01B60173
:102D200090E00E94C11731103A94F1E04F1A510817
:102D30004114510471F7E6C0843611F0893639F533
:102D4000F80127FF07C060817181828193810C5F48
:102D50001F4F08C060817181072E000C880B990BF2
:102D60000E5F1F4F2F76722E97FF09C090958095AA
:102D7000709561957F4F8F4F9F4F2068722E2AE08C
:102D800030E0A4010E94F117A82EA81844C085378E
:102D900029F42F7EB22E2AE030E025C0F22FF97FF1
:102DA000BF2E8F36C1F018F4883579F0B5C0803762
:102DB00019F0883721F0B0C02F2F2061B22EB4FE59
:102DC0000DC08B2D8460B82E09C024FF0AC09F2F30
:102DD0009660B92E06C028E030E005C020E130E062
:102DE00002C020E132E0F801B7FE07C060817181C6
:102DF000828193810C5F1F4F06C06081718180E0EA
:102E000090E00E5F1F4FA4010E94F117A82EA81892
:102E1000FB2DFF777F2E76FE0BC0372D3E7FA5144E
:102E200050F474FE0AC072FC08C0372D3E7E05C007
:102E3000BA2C372D03C0BA2C01C0B52C34FF0DC0FD
:102E4000FE01EA0DF11D8081803311F4397E09C045
:102E500032FF06C0B394B39404C0832F867809F080
:102E6000B39433FD13C030FF06C0B31498F43A0C8A
:102E7000532C5B1810C0B31470F4B60180E290E0DC
:102E80003C870E94C117B3943C85F5CFB31418F466
:102E90003B1802C05A2C312C34FF12C0B60180E31B
:102EA00090E03C870E94C1173C8532FF17C031FD7E
:102EB00003C088E790E002C088E590E0B6010CC04E
:102EC000832F867859F031FF02C08BE201C080E287
:102ED00037FD8DE2B60190E00E94C117A51438F4C9
:102EE000B60180E390E00E94C1175A94F7CFAA94EC
:102EF000F401EA0DF11D8081B60190E00E94C11736
:102F0000A110F5CF332009F450CEB60180E290E055
:102F10000E94C1173A94F6CFF6018681978102C0CC
:102F20008FEF9FEF2C960FB6F894DEBF0FBECDBF8C
:102F3000DF91CF911F910F91FF90EF90DF90CF9095
:102F4000BF90AF909F908F907F906F905F904F90C9
:102F50003F902F900895FC01059061507040011042
:102F6000D8F7809590958E0F9F1F0895FC016150B2
:102F7000704001900110D8F7809590958E0F9F1F9B
:102F800008950F931F93CF93DF93182F092FEB0111
:102F90008B8181FD03C08FEF9FEF1EC082FF0FC0AA
:102FA0002E813F818C819D812817390774F4E88137
:102FB000F981CF01019699838883108306C0E88543
:102FC000F985812F0995892B31F78E819F81019693
:102FD0009F838E83812F902FDF91CF911F910F912F
:102FE0000895FA01AA27283051F1203181F1E8949F
:102FF0006F936E7F6E5F7F4F8F4F9F4FAF4FB1E0EC
:103000003ED0B4E03CD0670F781F891F9A1FA11DE6
:10301000680F791F8A1F911DA11D6A0F711D811DE7
:10302000911DA11D20D009F468943F912AE0269FAC
:1030300011243019305D3193DEF6CF010895462F0B
:103040004770405D4193B3E00FD0C9F7F6CF462FEC
:103050004F70405D4A3318F0495D31FD4052419355
:1030600002D0A9F7EACFB4E0A69597958795779512
:103070006795BA95C9F700976105710508959B0199
:10308000AC010A2E06945795479537952795BA9522
:10309000C9F7620F731F841F951FA01D0895DC01DF
:1030A000CB01FC01F999FECF06C0F2BDE1BDF89A53
:1030B000319600B40D9241505040B8F70895F999F7
:1030C000FECF92BD81BDF89A992780B50895A6E1FB
:1030D000B0E044E050E00C945118DC01A40FB51F9F
:1030E0004150504048F0CB01840F951F2E910E9413
:1030F0007E1841505040D0F70895262FF999FECF01
:1031000092BD81BDF89A019700B4021639F01FBA3A
:1031100020BD0FB6F894FA9AF99A0FBE0895039657
:10312000272F0E947E180E947D18252F0E947E184E
:10313000242F0C947E180196272F0E947E180C9441
:063140007D18F894FFCF9A
:1031460000000001000000000000AE0000000000CA
:1031560000030000000016010701000020408080E7
:103166004001100836090036090036090026060116
:1031760036090023060336090036090036090036EB
:1031860009002006033609001D06031C0601360940
:10319600003609003609001B06011806031706014A
:1031A60016060136090036090036090036090036CA
:1031B60009003609003609001306031206010F0638
:1031C600030C06030B0601080603050603020603A5
:1031D600FF0503FC0503F90503F60503F30503F0F4
:1031E6000503EF0501EE0501ED0501EC0501EB0513
:1031F60001EA0501E90501E80501E70501E6050122
:10320600E50501E40501E30501E20501E10501E04B
:103216000501DF0501DE0501DB0503DA0501D7053A
:1032260003D40503D30501D00503CD0503CA050361
:10323600C70503C40503C10503BE0503BB0503B8E3
:103246000503B50503B20503AF0503AC0503A905E0
:1032560003A60503A30503A005039D05039A05031D
:103266009705039405039105038E05038B050388D3
:1032760005038505038205038105017E05037D059A
:10328600017C0501790503780501770501760501BD
:10329600750501740501730501720501710501705B
:1032A60005016F05016E05016D05016C05016B05D4
:1032B600016A0501690501680501670501660501E1
:1032C600650501640501630501620501610501608B
:1032D60005015F05015C0503590503560503530502
:1032E600035005033609004D05033609003609006B
:1032F6003609004C05014B05014A05014905014601
:1033060005034305034005033D05033A0503360956
:10331600003609003705033405033105032E05037E
:103326002D05012A05032705032405032105031E90
:1033360005031B05031805031505031205030F05F1
:10334600030C05030B050108050305050302050328
:10335600FF0403FC0403F90403F60403F30403F077
:103366000403ED0403EA0403E70403E40403E104AD
:1033760003DE0403DB0403D80403D50403D20403E9
:10338600CF0403CC0403C90403C60403C30403C067
:103396000403BD0403BA0403B70403B40403B1046D
:1033A60003AE0403AB0403AA0401A90401A80401A3
:1033B600A70401A60401A50401A40401A30401A213
:1033C6000401A10401A004019F04019E04019D04BF
:1033D600019C04019B04019A0401990401980401CB
:1033E6009704019604019504019404019304019243
:1033F60004019104018E04038B04038804038504ED
:10340600038204038104017E04037B04037804031E
:103416007504037204036F04036C040369040366F2
:1034260004036304036004035D04035A040357049E
:10343600035404035104034E04034B0403480403DA
:103446004504034204033F04033C040339040336E2
:1034560004033304033004032D04032A040327045E
:1034660003240403AFF66FAFE26FAFFA6FAFE26FFC
:10347600AFEA6FB9F579AFF46FAFF36FAFCB6FAF5C
:10348600D56FAFD46FAFEB6FAFC96FAFCA6FAFF188
:103496006FAFD16FAFCD6FAFE96FAFE16FAFD26FE7
:1034A600AFF76FAFD56FB9C679AFC66FAFE46FAF81
:1034B600C56FAFD36FAFF56FAFF26FAFCC6FAFEC39
:1034C6006FE7AFCE6FAFF66FB9E379AFDD6FB9C512
:1034D60079E1CBFAC9FBF3F2E9CAF7CDF4FCE4D5FE
:1034E600ECD4CCEBD3EAF1D2E2E3D1B9CE79AFE3B7
:1034F6006FAFE26FAFFA6FAFE26FAFEA6FB9F57910
:10350600AFF46FAFF36FAFCB6FAFD56FAFD46FAF15
:10351600EB6FAFC96FAFCA6FAFF16FAFD16FAFCD02
:103526006FAFE96FAFE16FAFD26FAFF76FAFD56F28
:10353600B9C679AFC66FAFE46FAFC56FAFD36FAF24
:10354600F56FAFF26FAFCC6FAFEC6FE797D95797C8
:10355600DB57B9D07997C257AFDB6FAFC36FAFDA1E
:103566006FAFC26FAFD96FAFC16FAFDF6FC0B9DEDC
:103576007997DC57B9F87997C757B9C879B9D8791F
:10358600B9F079B9E879B9E079D8F0E8E0AFC76F72
:10359600AFCE6FAFF66FB9E379AFDD6FB9C579E13D
:1035A600CBFAC9FBF3F2E9CAF7CDF4FCE4D5ECD4C7
:1035B600CCEBD3EAF1D2E2E3D1B9CE79CFF6B9D6E4
:1035C60079C6B9ED79B9E179B9CB79B9FA79B9C9D9
:1035D60079B9FB79B9F379B9F279B9E979B9CA79DF
:1035E600B9F779B9CD79B9F479B9FC79B9E479B98A
:1035F600D579B9EC79B9D479B9CC79B9EB79B9D3AC
:1036060079B9EA79B9F179B9D279B9E279B9E379CF
:10361600B9D179F5B9FE79B9E579EEB9FD79D6ED85
:10362600C4DBC3DAC2D9C1DFC7DCFEE5DDFDC5CE2A
:10363600B9C479B9DB79B9C379B9DA79B9C279B9D3
:10364600D979B9C179B9DF79B9C779E797C35797F6
:10365600DA57D097C157C0DE97C457F8C8B9DE7994
:10366600B9C87997DF57FFB80F3412CDABB0B000A9
:103676000101010102FCFDFEFF1CCFFF5A0000758F
:103686000A200060406040000C0A202A2A2A2A2AC2
:10369600206B65796D616E36342076657273696F5D
:1036A6006E20312E35207265616479202A2A2A2AF5
:1036B6002A0A0A202020206E6F20636F6E666967D3
:1036C60075726174696F6E20666F756E6420696EBF
:1036D60020656570726F6D0A20202020202075738A
:1036E600696E672066616C6C6261636B20636F6EE6
:1036F60066696775726174696F6E0A0A20202020F8
:103706002020205F763A2074797065206669726D94
:10371600776172652076657273696F6E0A20202064
:10372600202020205F623A20656E74657220626FE9
:103736006F746C6F616465720A202020202020203F
:103746005F663A2074657374206372797374616C72
:10375600206672657175656E63790A2020202020C7
:1037660020205F743A20747970652074686973202C
:103776006D6573736167650A0A72656164792E0AFD
:10378600000C0A202A2A2A2A2A20206B65796D61D4
:103796006E3634206672657175656E637920746560
:1037A600737420202A2A2A2A2A0A0A69662074683B
:1037B6006520666F6C6C6F77696E672074656E2026
:1037C600646F747320617265206E6F7420747970F3
:1037D60065640A776974682061626F7574206F6E1C
:1037E60065207365636F6E642064656C617920691A
:1037F6006E206265747765656E2C0A636865636B17
:103806002061746D656C20667573657320616E64E6
:103816002F6F72206372797374616C2063697263AF
:103826007569740A006669726D7761726520312E5A
:10383600352046656220323120323031372031342E
:103846003A34323A343500303030303030303000AF
:10385600612025730A00622025730A0A002A007374
:10386600657400636C656172656400656E7465728B
:10387600206E65772070617373776F72643A2000EB
:10388600726570656174206E6577207061737377F9
:103896006F72643A20006F6B2C2070617373776FC0
:1038A60072642025730A0A0070617373776F7264FD
:1038B60073206469666665722C206E6F7468696E23
:1038C60067206368616E6765640A0A006E6F207020
:1038D600617373776F726420646566696E65640AE6
:0238E6000A00D6
:020000021000EC
:10E000007EC00000BFC00000A3C00000A1C000008F
:10E010009FC000009DC000009BC0000099C0000090
:10E0200097C0000095C0000093C0000091C00000A0
:10E030008FC000008DC000008BC0000089C00000B0
:10E0400087C0000085C0000083C0000081C00000C0
:10E050007FC000007DC000007BC0000079C00000D0
:10E0600077C0000075C0000073C0000071C00000E0
:10E070006FC000006DC000006BC0000069C00000F0
:10E0800067C0000065C0000063C00000BBBEEC2D8F
:10E09000FD2DB7B6B0FCFDCF27BFE895B7B6B0FCF5
:10E0A000FDCF21E1B7B6B6FCF4CF08950902120006
:10E0B000010100803209040000000000000012018C
:10E0C0001001FF000008C016DC050201010200017A
:10E0D0000E035500530042006100730070001C03E2
:10E0E0007700770077002E006600690073006300F8
:10E0F00068006C002E00640065000403090411240C
:10E100001FBECFEFD0E4DEBFCDBF24B7D0E4CEEF4B
:10E110003991303F399109F03FEF30933E01209320
:10E120003D0111E0A0E0B1E0ECEBF9EE01E00BBF46
:10E1300002C007900D92A630B107D9F721E0A6E002
:10E14000B1E001C01D92AD33B207E1F78CD134C408
:10E1500057CFA82FB92F80E090E041E050EA6095BA
:10E1600030E009C02D9182279795879510F084277C
:10E170009527305EC8F36F5FA8F30895EADF8D93AB
:10E180009D930895CF93CFB7CF93DF93C395499BCA
:10E19000E9F7499B0BC0499B09C0499B07C0499BB4
:10E1A00005C0499B03C0499B01C089C06F93C091C2
:10E1B0002001DD27C95DDE4F2F9365E5499B03C034
:10E1C0002F916F91E6CF0F931F934F9320E040E183
:10E1D0005F9309B1067001FB27F93F9350E03BE0E4
:10E1E00039C0167040642F77012F5F5F1EC04068F2
:10E1F00019B116702F7752501FC0406409B12F77A4
:10E200000670D1F15F5F00C023C0406219B12F7763
:10E21000167091F15F5F00C025C006701027515045
:10E2200012F45D5F0000115027952C3F19B1C8F61C
:10E2300016700127015027952C3FC8F642274993B5
:10E2400009B1067010274F73115027952C3FA8F67F
:10E250004695469519B1167079F00127015027951A
:10E260002C3F98F66B5A60F3315009B1B0F600C0FC
:10E2700011E01CBB002717C03B503195C31BD04099
:10E2800011E01CBB0881033CF9F00B34E9F020914C
:10E290001E011981110F1213EDCF093651F10D3204
:10E2A00011F0013E39F7009325013F915F914F91A5
:10E2B0001F910F912F916F91CCB3C0FD67CFDF916C
:10E2C000CF91CFBFCF91189520912501222369F3DB
:10E2D00010912301112339F534303AF130932301A1
:10E2E00020931F01109120013BE0311B309320014E
:10E2F0001CC0009123010130B4F40AE53091010102
:10E3000034FD14C000930101C3E1D1E013C005271F
:10E3100010E000C000000BB91AC0052710E0221F52
:10E320001DC010E021C04AE502C032ED432FC4E118
:10E33000D0E032E01AB11660599A0BB11AB956E022
:10E3400020E865E320FF05270BB9279517951C3FAB
:10E35000F0F66695B8F7B1F720FF05270BB92795BA
:10E3600017951C3FD0F62795179517FF0527000036
:10E370001C3F0BB9B0F629913A9519F7097F109116
:10E380002401110FC651D0400BB911F010931E019A
:10E3900011E01CBB02601AB1197F402F497F54E085
:10E3A0005A95F1F70BB91AB94BB97FCFDC01139627
:10E3B0003C911397F32F14962C911497E22F1296F9
:10E3C0009C911297903339F42370E22FF0E0EE5FC6
:10E3D000FE4F80810895983529F431110EC0E1E097
:10E3E000F0E006C0903599F431110CC0E0E0F0E0A7
:10E3F00089E08093570084910895383091F5E3E0E7
:10E40000F0E0F6CF383069F5E2E0F0E0F1CF90329D
:10E4100041F4CF01A0E0B0E0880F991FAA1FBB1FF5
:10E420000CC0983271F4CF01A0E0B0E0880F991FC2
:10E43000AA1FBB1F0196A11DB11DABBFFC01879197
:10E440000895903A11F4CF0189C2903C29F41596B1
:10E450006C91CF0190D205C09F3F19F481EF80935A
:10E46000110180E008951AB881E08BB985BF92E070
:10E4700095BFE0E0F1E7A89531979040E1F704B649
:10E4800003FE0EC08EEF9FE071D2C1E0803B904B47
:10E4900009F0C0E06FEF7FEF8EEF9FE07AD208C007
:10E4A00004B601FE04C0C9B1C170C82701C0C0E0F4
:10E4B00014BEC1110CC0F894519A1BB81DBA109229
:10E4C000690081E085BF15BEE0E0F0E009958EEFC0
:10E4D0008093110114BE0FB6F894A8958091600046
:10E4E000886180936000109260000FBE8091690087
:10E4F000826080936900E89A519A8CE0E0E0F5E34D
:10E50000A89531978040E1F75198789481EF8093F6
:10E51000110110912301135017FD74C18091200146
:10E52000CCE0D0E0C81BD109C95DDE4F80911F014E
:10E530008D3209F0C0C0183009F062C183EC8093BD
:10E5400013018AE580930101109212013881832F13
:10E5500080769981882309F43FC046E051E05093CA
:10E56000220140932101933031F4CE011FDF8093CB
:10E57000090184E096C0953009F492C09A3009F4FC
:10E580008FC08CEF890F8630E0F44A815B81509315
:10E590000E0140930D01993039F48C819D81909347
:10E5A000100180930F0114C08E8180930C012D8186
:10E5B000227020930B0190930A0137FD6DC08FEFFD
:10E5C0006BC080911101923029F48E7F80931101EC
:10E5D00080E067C08160FACF8A8110921C0191119E
:10E5E00006C010921D012CE131E082E050C0953050
:10E5F00019F4809324013DC09630A9F59B81913098
:10E6000019F48EEB90EE04C0923041F48CEA90EE57
:10E61000909322018093210182E121C09330F1F493
:10E62000811108C08AEF90EE90932201809321011E
:10E6300084E015C0813041F48EED90EE909322017C
:10E64000809321018CE10BC0823041F480ED90EE8B
:10E6500090932201809321018EE001C080E090E43C
:10E66000909312011EC0983079F0993031F4809364
:10E6700026012CE131E080E00AC081E09A3009F007
:10E6800080E02CE131E003C026E231E081E030930C
:10E6900022012093210105C090E89093120108C047
:10E6A00081E09F81911104C09E81981708F4892F01
:10E6B00080930001A5C08091120187FFA1C0009145
:10E6C0000C01011708F4102F011B00930C01F12C11
:10E6D000F11608F091C080910A018730A0F06E0118
:10E6E000FFEFCF1ADF0A688180910D0190910E0132
:10E6F0009C012F5F3F4F30930E0120930D013BD1C2
:10E70000F394E601E5CF80910D0190910E01A09167
:10E710000F01B09110018115904EA140B10508F094
:10E720006DC0F394F394F89440910D0150910E0153
:10E7300060910F01709110012991399181E00901D7
:10E74000FA0160935B0080935700E8951124789458
:10E7500080910D0190910E01A0910F01B0911001D7
:10E760000296A11DB11D80930D0190930E01A093FF
:10E770000F01B0931001882351F00111A9CFF116B8
:10E7800008F4A6CF80910B01882309F4A1CFF89457
:10E7900080910D0190910E01A0910F01B091100197
:10E7A0000297A109B10923E0FC01A0935B0020932B
:10E7B0005700E895789407B600FCFDCFF894809157
:10E7C0000D0190910E01A0910F01B09110010297DF
:10E7D000A109B10925E0FC01A0935B00209357003B
:10E7E000E895789407B600FCFDCFF89481E180931A
:10E7F0005700E89578946CCF011102C01092000187
:10E80000109223018091010184FF7EC0809100015C
:10E810008F3F09F479C0C82F893008F0C8E08C1BFD
:10E82000809300019091130188E889278093130158
:10E83000CC2309F48DC08091120187FF37C08091ED
:10E840000C018C1708F4C82F8C1B80930C01B0901E
:10E850000A01D0E004E111E0CD1709F449C0C090ED
:10E860000D01D0900E01E0900F01F090100186E0B4
:10E870008B1530F480910D0190910E016FD003C083
:10E88000EBBEF6018791F80180830F5F1F4FFFEF0A
:10E89000CF1ADF0AEF0AFF0AC0920D01D0920E01D3
:10E8A000E0920F01F0921001DF5FD6CFA09121011D
:10E8B000B091220186FF11C024E131E08C2FAD011F
:10E8C00060E070E061606BBFFA014791F90141932C
:10E8D0009F011196815099F707C0E4E1F1E08C2F78
:10E8E0009D9191938150E1F7B0932201A093210172
:10E8F0006C2F84E191E042DCCC5FCC3019F08FEFDB
:10E9000080930001C093010184E199B1967031F4C4
:10E910008150D9F71092240110921E0180911101AB
:10E92000803130F0489B0FC080911101805109C0A7
:10E93000489909C080911101823028F0809111011D
:10E94000825080931101809111018111E2CDB3CDEC
:10E9500060E084E191E012DCC4E0D1CFF999FECF10
:10E9600092BD81BDF89A992780B50895A8E1B0E0DD
:10E9700042E050E013C0262FF999FECF1FBA92BD96
:10E9800081BD20BD0FB6F894FA9AF99A0FBE019690
:10E990000895F1DF272FF0CFDC01CB01FC01F999BD
:10E9A000FECF06C0F2BDE1BDF89A319600B40D92DB
:0CE9B00041505040B8F70895F894FFCF94
:06E9BC00FF5A1E97050042
:040000031000E00009
:00000001FF
